:020000040800F2
:1000000000C00020AD5C0008815C0008855C000831
:10001000895C00088D5C0008915C0008000000000D
:10002000000000000000000000000000955C0008D7
:10003000995C0008000000009D5C0008A15C0008BD
:10004000FD5C0008FD5C0008FD5C0008FD5C00082C
:10005000FD5C0008FD5C0008FD5C0008FD5C00081C
:10006000FD5C0008FD5C0008FD5C0008794B0008A1
:10007000FD5C0008FD5C0008FD5C0008FD5C0008FC
:10008000FD5C0008FD5C0008FD5C0008FD5C0008EC
:10009000FD5C0008FD5C0008FD5C0008FD5C0008DC
:1000A000FD5C0008FD5C0008FD5C0008FD5C0008CC
:1000B000FD5C0008FD5C0008FD5C0008FD5C0008BC
:1000C000FD5C0008FD5C0008FD5C0008FD5C0008AC
:1000D000FD5C0008FD5C0008FD5C0008FD5C00089C
:1000E000FD5C0008FD5C0008FD5C0008FD5C00088C
:1000F000FD5C0008FD5C0008FD5C0008FD5C00087C
:10010000FD5C0008FD5C0008FD5C0008FD5C00086B
:10011000FD5C0008FD5C0008FD5C0008FD5C00085B
:10012000FD5C0008FD5C0008FD5C0008FD5C00084B
:1001300000000000000000000000000000000000BF
:1001400000000000000000000000000000000000AF
:10015000000000000000000000000000000000009F
:10016000000000000000000000000000000000008F
:10017000000000000000000000000000000000007F
:10018000000000000000000000000000000000006F
:10019000000000000000000000000000000000005F
:1001A000000000000000000000000000000000004F
:1001B000000000000000000000000000000000003F
:1001C000000000000000000000000000000000002F
:1001D000000000000000000000000000000000001F
:0401E0005FF8E0F1F3
:1001E80010B5054C237833B9044B13B10448AFF369
:1001F80000800123237010BD500000200000000083
:10020800605D000808B5064B1BB106480649AFF308
:1002180000800648036813B1054B03B1984708BD31
:1002280000000000605D0008540000204C00002021
:100238000000000081F0004102E000BF83F00043AD
:1002480030B54FEA41044FEA430594EA050F08BF69
:1002580090EA020F1FBF54EA000C55EA020C7FEA2D
:10026800645C7FEA655C00F0E2804FEA5454D4EBAA
:100278005555B8BF6D420CDD2C4480EA020281EA74
:10028800030382EA000083EA010180EA020281EAAC
:100298000303362D88BF30BD11F0004F4FEA0131FE
:1002A8004FF4801C4CEA113102D0404261EB41010D
:1002B80013F0004F4FEA03334CEA133302D0524293
:1002C80063EB430394EA050F00F0A780A4F101044F
:1002D800D5F1200E0DDB02FA0EFC22FA05F2801889
:1002E80041F1000103FA0EF2801843FA05F359416F
:1002F8000EE0A5F120050EF1200E012A03FA0EFCEE
:1003080028BF4CF0020C43FA05F3C01851EBE37117
:1003180001F0004507D54FF0000EDCF1000C7EEB34
:1003280000006EEB0101B1F5801F1BD3B1F5001F72
:100338000CD349085FEA30004FEA3C0C04F1010491
:100348004FEA445212F5800F80F09A80BCF1004FBA
:1003580008BF5FEA500C50F1000041EB045141EA3C
:10036800050130BD5FEA4C0C404141EB010111F43D
:10037800801FA4F10104E9D191F0000F04BF0146E8
:100388000020B1FA81F308BF2033A3F10B03B3F1C6
:1003980020020CDA0C3208DD02F1140CC2F10C0256
:1003A80001FA0CF021FA02F10CE002F11402D8BFB4
:1003B800C2F1200C01FA02F120FA0CFCDCBF41EA80
:1003C8000C019040E41AA2BF01EB0451294330BD4F
:1003D8006FEA04041F3C1CDA0C340EDC04F114042C
:1003E800C4F1200220FA04F001FA02F340EA030003
:1003F80021FA04F345EA030130BDC4F10C04C4F149
:10040800200220FA02F001FA04F340EA0300294628
:1004180030BD21FA04F0294630BD94F0000F83F472
:10042800801306BF81F480110134013D4EE77FEA55
:10043800645C18BF7FEA655C29D094EA050F08BFA1
:1004480090EA020F05D054EA000C04BF1946104682
:1004580030BD91EA030F1EBF0021002030BD5FEAC6
:10046800545C05D14000494128BF41F0004130BDEE
:1004780014F580043CBF01F5801130BD01F0004542
:1004880045F0FE4141F470014FF0000030BD7FEAB5
:10049800645C1ABF194610467FEA655C1CBF0B46B0
:1004A800024650EA013406BF52EA033591EA030FC7
:1004B80041F4002130BD00BF90F0000F04BF0021BF
:1004C800704730B54FF4806404F132044FF00005F2
:1004D8004FF0000150E700BF90F0000F04BF00216B
:1004E800704730B54FF4806404F1320410F00045D1
:1004F80048BF40424FF000013EE700BF42004FEACC
:10050800E2014FEA31014FEA02701FBF12F07F4348
:1005180093F07F4F81F06051704792F0000F14BF45
:1005280093F07F4F704730B54FF4607401F0004589
:1005380021F0004120E700BF50EA010208BF7047E0
:1005480030B54FF000050AE050EA010208BF7047D5
:1005580030B511F0004502D5404261EB41014FF43E
:10056800806404F132045FEA915C3FF4DCAE4FF042
:1005780003025FEADC0C18BF03325FEADC0C18BF29
:10058800033202EBDC02C2F1200300FA03FC20FA7A
:1005980002F001FA03FE40EA0E0021FA02F11444C7
:1005A800C1E600BF70B54FF0FF0C4CF4E06C1CEADC
:1005B80011541DBF1CEA135594EA0C0F95EA0C0F51
:1005C80000F0DEF82C4481EA030621EA4C5123EAC4
:1005D8004C5350EA013518BF52EA033541F48011F3
:1005E80043F4801338D0A0FB02CE4FF00005E1FBA6
:1005F80002E506F00042E0FB03E54FF00006E1FBF0
:1006080003569CF0000F18BF4EF0010EA4F1FF0432
:10061800B6F5007F64F5407404D25FEA4E0E6D4172
:1006280046EB060642EAC62141EA55514FEAC52083
:1006380040EA5E504FEACE2EB4F1FD0C88BFBCF5FF
:10064800E06F1ED8BEF1004F08BF5FEA500E50F1B0
:10065800000041EB045170BD06F0004646EA010176
:1006680040EA020081EA0301B4EB5C04C2BFD4EBA8
:100678000C0541EA045170BD41F480114FF0000EA1
:10068800013C00F3AB8014F1360FDEBF002001F00F
:10069800004170BDC4F10004203C35DA0C341BDC89
:1006A80004F11404C4F1200500FA05F320FA04F05B
:1006B80001FA05F240EA020001F0004221F000418F
:1006C80010EBD37021FA04F642EB06015EEA430E02
:1006D80008BF20EAD37070BDC4F10C04C4F1200532
:1006E80000FA04F320FA05F001FA04F240EA0200E5
:1006F80001F0004110EBD37041F100015EEA430EB6
:1007080008BF20EAD37070BDC4F1200500FA05F2D5
:100718004EEA020E20FA04F301FA05F243EA020354
:1007280021FA04F001F0004121FA04F220EA020063
:1007380000EBD3705EEA430E08BF20EAD37070BDA9
:1007480094F0000F0FD101F00046400041EB010189
:1007580011F4801F08BF013CF7D041EA060195F06B
:10076800000F18BF704703F00046520043EB030325
:1007780013F4801F08BF013DF7D043EA0603704712
:1007880094EA0C0F0CEA135518BF95EA0C0F0CD01D
:1007980050EA410618BF52EA4306D1D181EA030163
:1007A80001F000414FF0000070BD50EA410606BF5D
:1007B8001046194652EA430619D094EA0C0F02D1A2
:1007C80050EA013613D195EA0C0F05D152EA0336E7
:1007D8001CBF104619460AD181EA030101F0004105
:1007E80041F0FE4141F470014FF0000070BD41F04E
:1007F800FE4141F4780170BD70B54FF0FF0C4CF428
:10080800E06C1CEA11541DBF1CEA135594EA0C0F46
:1008180095EA0C0F00F0A7F8A4EB050481EA030E93
:1008280052EA03354FEA013100F088804FEA03337A
:100838004FF0805545EA131343EA12634FEA022248
:1008480045EA111545EA10654FEA00260EF0004109
:100858009D4208BF964244F1FD0404F5407402D25B
:100868005B084FEA3202B61A65EB03055B084FEAEC
:1008780032024FF480104FF4002CB6EB020E75EBE9
:10088800030E22BFB61A754640EA0C005B084FEA11
:100898003202B6EB020E75EB030E22BFB61A75468E
:1008A80040EA5C005B084FEA3202B6EB020E75EBD9
:1008B800030E22BFB61A754640EA9C005B084FEA51
:1008C8003202B6EB020E75EB030E22BFB61A75465E
:1008D80040EADC0055EA060E18D04FEA051545EA4D
:1008E80016754FEA06164FEAC30343EA52734FEAF6
:1008F800C2025FEA1C1CC0D111F4801F0BD141EA6F
:1009080000014FF000004FF0004CB6E711F4801FD3
:1009180004BF01430020B4F1FD0C88BFBCF5E06FB3
:100928003FF6AFAEB5EB030C04BFB6EB020C5FEAC3
:10093800500C50F1000041EB045170BD0EF0004E18
:100948004EEA113114EB5C04C2BFD4EB0C0541EA4A
:10095800045170BD41F480114FF0000E013C90E647
:1009680045EA060E8DE60CEA135594EA0C0F08BF0B
:1009780095EA0C0F3FF43BAF94EA0C0F0AD150EA0A
:1009880001347FF434AF95EA0C0F7FF425AF10469D
:1009980019462CE795EA0C0F06D152EA03353FF4C5
:1009A800FDAE1046194622E750EA410618BF52EA42
:1009B80043067FF4C5AE50EA41047FF40DAF52EA16
:1009C80043057FF4EBAE12E74FF0FF3C06E000BFB3
:1009D8004FF0010C02E000BF4FF0010C4DF804CDC0
:1009E8004FEA410C7FEA6C5C4FEA430C18BF7FEA80
:1009F8006C5C1BD001B050EA410C0CBF52EA430CAE
:100A080091EA030F02BF90EA020F0020704710F12D
:100A1800000F91EA030F58BF994208BF90422CBFBC
:100A2800D8176FEAE37040F0010070474FEA410CB5
:100A38007FEA6C5C02D150EA013C07D14FEA430CD3
:100A48007FEA6C5CD6D152EA033CD3D05DF8040B44
:100A5800704700BF8446104662468C461946634676
:100A680000E000BF01B5FFF7B7FF002848BF10F14D
:100A7800000F01BD4DF808EDFFF7F4FF0CBF012092
:100A880000205DF808FB00BF4DF808EDFFF7EAFF0E
:100A980034BF012000205DF808FB00BF4DF808EDC9
:100AA800FFF7E0FF94BF012000205DF808FB00BFBE
:100AB8004DF808EDFFF7CEFF94BF012000205DF848
:100AC80008FB00BF4DF808EDFFF7C4FF34BF012055
:100AD80000205DF808FB00BF4FEA410212F5001242
:100AE80015D211D56FF47873B3EB625212D94FEA6D
:100AF800C12343F0004343EA505311F0004F23FA57
:100B080002F018BF404270474FF00000704750EAAB
:100B1800013005D111F0004008BF6FF00040704768
:100B28004FF00000704700BF4A0011D212F50012C2
:100B380011D20DD56FF47873B3EB62520ED44FEA2D
:100B4800C12343F0004343EA505323FA02F07047AD
:100B58004FF00000704750EA013002D14FF0FF30EB
:100B680070474FF0000070474FEA4102B2F1E0438E
:100B780024BFB3F5001CDCF1FE5C0DD901F0004C7C
:100B88004FEAC0024CEA5070B2F1004F40EB8300CC
:100B980008BF20F00100704711F0804F21D113F1F8
:100BA8003872BCBF01F00040704741F480114FEA31
:100BB8005252C2F11802C2F1200C10FA0CF320FABA
:100BC80002F018BF40F001004FEAC1234FEAD323D7
:100BD80003FA0CFC40EA0C0023FA02F34FEA430341
:100BE800CCE77FEA625307D150EA01331EBF4FF0CA
:100BF800FE4040F44000704701F0004040F0FE40E5
:100C080040F40000704700BF80F0004002E000BFE1
:100C180081F0004142001FBF5FEA410392EA030FDF
:100C28007FEA226C7FEA236C6AD04FEA1262D2EB29
:100C38001363C1BFD218414048404140B8BF5B422E
:100C4800192B88BF704710F0004F40F4000020F0C7
:100C58007F4018BF404211F0004F41F4000121F0DD
:100C68007F4118BF494292EA030F3FD0A2F1010227
:100C780041FA03FC10EB0C00C3F1200301FA03F165
:100C880000F0004302D5494260EB4000B0F5000F88
:100C980013D3B0F1807F06D340084FEA310102F147
:100CA8000102FE2A51D2B1F1004F40EBC25008BFF9
:100CB80020F0010040EA03007047490040EB0000C3
:100CC80010F4000FA2F10102EDD1B0FA80FCACF1F2
:100CD800080CB2EB0C0200FA0CF0AABF00EBC250F1
:100CE80052421843BCBFD0401843704792F0000FDF
:100CF80081F4000106BF80F400000132013BB5E732
:100D08004FEA41037FEA226C18BF7FEA236C21D0A7
:100D180092EA030F04D092F0000F08BF084670470C
:100D280090EA010F1CBF0020704712F07F4F04D1DA
:100D3800400028BF40F00040704712F100723CBFED
:100D480000F50000704700F0004343F0FE4040F417
:100D5800000070477FEA226216BF08467FEA2363D5
:100D68000146420206BF5FEA412390EA010F40F4C0
:100D7800800070474FF0000304E000BF10F000430C
:100D880048BF40425FEA000C08BF704743F09643F3
:100D980001464FF000001CE050EA010208BF70470E
:100DA8004FF000030AE000BF50EA010208BF704795
:100DB80011F0004302D5404261EB41015FEA010CAA
:100DC80002BF84460146002043F0B64308BFA3F1A2
:100DD8008053A3F50003BCFA8CF2083AA3EBC25384
:100DE80010DB01FA02FC634400FA02FCC2F12002A3
:100DF800BCF1004F20FA02F243EB020008BF20F0DA
:100E08000100704702F1200201FA02FCC2F120023F
:100E180050EA4C0021FA02F243EB020008BF20EA34
:100E2800DC7070474FF0FF0C1CEAD0521EBF1CEA62
:100E3800D15392EA0C0F93EA0C0F6FD01A4480EA50
:100E4800010C400218BF5FEA41211ED04FF0006339
:100E580043EA501043EA5111A0FB01310CF0004065
:100E6800B1F5000F3EBF490041EAD3715B0040EA8B
:100E7800010062F17F02FD2A1DD8B3F1004F40EB5B
:100E8800C25008BF20F00100704790F0000F0CF02E
:100E9800004C08BF49024CEA502040EA51207F3AF2
:100EA800C2BFD2F1FF0340EAC250704740F40000CD
:100EB8004FF00003013A5DDC12F1190FDCBF00F0BE
:100EC80000407047C2F10002410021FA02F1C2F16C
:100ED800200200FA02FC5FEA310040F1000053EA08
:100EE8004C0308BF20EADC70704792F0000F00F056
:100EF800004C02BF400010F4000F013AF9D040EA5C
:100F08000C0093F0000F01F0004C02BF490011F4EF
:100F1800000F013BF9D041EA0C018FE70CEAD153ED
:100F280092EA0C0F18BF93EA0C0F0AD030F0004C6D
:100F380018BF31F0004CD8D180EA010000F0004021
:100F4800704790F0000F17BF90F0004F084691F0DF
:100F5800000F91F0004F14D092EA0C0F01D1420219
:100F68000FD193EA0C0F03D14B0218BF084608D1E2
:100F780080EA010000F0004040F0FE4040F400002C
:100F8800704740F0FE4040F4400070474FF0FF0CBF
:100F98001CEAD0521EBF1CEAD15392EA0C0F93EA06
:100FA8000C0F69D0A2EB030280EA010C49024FEA58
:100FB800402037D04FF0805343EA111143EA101311
:100FC8000CF000408B4238BF5B0042F17D024FF4C9
:100FD800000C8B4224BF5B1A40EA0C00B3EB510FA4
:100FE80024BFA3EB510340EA5C00B3EB910F24BF8D
:100FF800A3EB910340EA9C00B3EBD10F24BFA3EB12
:10100800D10340EADC001B0118BF5FEA1C1CE0D1D9
:10101800FD2A3FF650AF8B4240EBC25008BF20F08C
:10102800010070470CF0004C4CEA50207F32C2BFE0
:10103800D2F1FF0340EAC250704740F400004FF07D
:101048000003013A37E792F0000F00F0004C02BFAE
:10105800400010F4000F013AF9D040EA0C0093F078
:10106800000F01F0004C02BF490011F4000F013BD2
:10107800F9D041EA0C0195E70CEAD15392EA0C0F3A
:1010880008D142027FF47DAF93EA0C0F7FF470AF72
:10109800084676E793EA0C0F04D14B023FF44CAFB5
:1010A80008466EE730F0004C18BF31F0004CCAD14A
:1010B80030F000427FF45CAF31F000437FF43CAF86
:1010C8005FE700BF4FF0FF3C06E000BF4FF0010CA8
:1010D80002E000BF4FF0010C4DF804CD4FEA40028A
:1010E8004FEA41037FEA226C18BF7FEA236C11D0D4
:1010F80001B052EA530C18BF90EA010F58BFB2EB87
:10110800030088BFC81738BF6FEAE17018BF40F006
:10111800010070477FEA226C02D15FEA402C05D1BA
:101128007FEA236CE4D15FEA412CE1D05DF8040B3F
:10113800704700BF844608466146FFE70FB5FFF7D2
:10114800C9FF002848BF10F1000F0FBD4DF808ED8A
:10115800FFF7F4FF0CBF012000205DF808FB00BF7B
:101168004DF808EDFFF7EAFF34BF012000205DF8D5
:1011780008FB00BF4DF808EDFFF7E0FF94BF012022
:1011880000205DF808FB00BF4DF808EDFFF7D2FF1F
:1011980094BF012000205DF808FB00BF4DF808ED62
:1011A800FFF7C8FF34BF012000205DF808FB00BF2F
:1011B8004FEA4002B2F1FE4F0FD34FF09E03B3EB5C
:1011C80012620DD94FEA002343F0004310F0004F9C
:1011D80023FA02F018BF404270474FF000007047F2
:1011E80012F1610F01D1420205D110F0004008BF91
:1011F8006FF0004070474FF00000704742000ED279
:10120800B2F1FE4F0BD34FF09E03B3EB126209D439
:101218004FEA002343F0004323FA02F070474FF0EF
:101228000000704712F1610F01D1420202D14FF064
:10123800FF3070474FF00000704700BF0022044B9A
:10124800DA61044B1A6942F001021A6101807047A1
:10125800B800002000200240154BDB6813F0100F87
:1012680006D0144BDA6942F00202DA61102300E07A
:1012780000230F4AD26812F0040F06D00D4AD16934
:1012880041F00101D16143F00403094AD26912F027
:10129800010F09D0074AD16941F00401D161044A1C
:1012A800D16921F00101D161014AD360704700BFC3
:1012B80000200240B8000020074B1B6913F0800F84
:1012C80007D0054B054A5A6002F188325A6000205F
:1012D80070470120704700BF002002402301674586
:1012E800034B1A6942F080021A610020704700BF60
:1012F8000020024070B5044601F0A4F90646184DD6
:1013080008E0B4F1FF3F05D01CB301F09BF9801B46
:10131800A04220D8EB6813F0010FF2D1104BDB6824
:1013280013F0200F02D020220D4BDA600C4BDB6843
:1013380013F0100F09D10A4BDB6913F0010F04D128
:10134800074BDB6813F0040F07D0FFF785FF012078
:1013580070BD032070BD032070BD002070BD00BFAC
:10136800002002402DE9F84F80468A4616461F465F
:10137800264B1B7E012B46D00122244B1A764CF2B9
:101388005030FFF7B7FF0346B8BBB8F1010F05D0DF
:10139800B8F1020F05D14FF0020B04E04FF0010B3A
:1013A80001E04FF0040B4FF00008DFF8649022E0F2
:1013B8004FEA0813C3F12001A3F1200226FA03F42F
:1013C80007FA01F10C4327FA02F214430AEB48002A
:1013D800A1B2FFF733FF4CF25030FFF78BFFD9F87B
:1013E800103023F00103C9F81030034628B908F17A
:1013F80001085FFA88F8D845DAD30021034A117644
:101408001846BDE8F88F0220BDE8F88FB800002024
:101418000020024082B0084B1A68084BA3FB021355
:101428005B0A00FB03F0019000BF019B5A1E01926A
:10143800002BF9D102B0704700000020D34D621094
:101448002DE9F04182B00446036813F0010F6ED015
:10145800A24B5B6803F00C03042B0AD09F4B5B681C
:1014680003F00C03082B0DD19C4B5B6813F4803FF1
:1014780008D09A4B1B6813F4003F58D06368002BC0
:1014880055D1C1E16368B3F5803F08D103F18043CA
:1014980003F588331A6842F480321A6026E063B98B
:1014A80003F1804303F504331A6822F480321A608A
:1014B8001A6822F480221A6018E0B3F5A02F0CD124
:1014C80003F18043A3F53C331A6842F480221A6082
:1014D8001A6842F480321A6008E0804B1A6822F4D5
:1014E80080321A601A6822F480221A6063687BB11D
:1014F80001F0A8F80646794D05E001F0A3F8801B35
:10150800642800F283812B6813F4003FF5D00EE0C5
:1015180001F098F80646714D05E001F093F8801B3C
:10152800642800F275812B6813F4003FF5D1236815
:1015380013F0020F50D0694B5B6813F00C0F0AD000
:10154800664B5B6803F00C03082B16D1634B5B6892
:1015580013F4803F11D1614B1B6813F0020F03D0C5
:101568002369012B40F056815C4B196821F0F80182
:10157800626941EAC2021A602EE02369D3B10122EE
:10158800574B1A6001F05EF80646544D05E001F02D
:1015980059F8801B022800F23F812B6813F0020FD4
:1015A800F5D04E4B196821F0F801626941EAC20290
:1015B8001A6011E000224A4B1A6001F043F806460F
:1015C800464D05E001F03EF8801B022800F2268116
:1015D8002B6813F0020FF5D1236813F0080F29D0F8
:1015E800A369ABB101223F4B1A6001F02BF8064604
:1015F8003A4D05E001F026F8801B022800F2108120
:101608006B6A13F0020FF5D00120FFF703FF11E01A
:101618000022344B1A6001F015F806462F4D05E0FC
:1016280001F010F8801B022800F2FC806B6A13F0AE
:10163800020FF5D1236813F0040F00F08C80274BBC
:10164800DB6913F0805F0BD1244BDA6942F08052DA
:10165800DA61DB6903F080530193019B012500E007
:101668000025214B1B6813F4807F13D11E4B1A6889
:1016780042F480721A6000F0E5FF07461A4E05E052
:1016880000F0E0FFC01B642800F2CE80336813F43A
:10169800807FF5D0E368012B05D1104B1A6A42F020
:1016A80001021A622BE063B903F1804303F50433A6
:1016B8001A6A22F001021A621A6A22F004021A62F5
:1016C8001DE0052B12D1054B1A6A42F004021A627A
:1016D8001A6A42F001021A6211E000BF00100240CB
:1016E800000042428004424200700040574B1A6A90
:1016F80022F001021A621A6A22F004021A62E368EE
:1017080093B100F09FFF8046504E41F2883706E0C3
:1017180000F098FFC8EB0000B84200F28780336AF7
:1017280013F0020FF4D010E000F08CFF8046474E13
:1017380041F2883705E000F085FFC8EB0000B842A9
:1017480076D8336A13F0020FF5D125B13F4BDA6929
:1017580022F08052DA61E369002B6BD03B4A526871
:1017680002F00C02082A67D0022B3AD10022384B2B
:101778001A6000F067FF0646344D04E000F062FF8F
:10178800801B02285AD82B6813F0007FF6D1236AF1
:10179800B3F5803F09D103F1804303F588335968D5
:1017A80021F40031A2680A435A60284B596821F491
:1017B8007411206A626A02430A435A600122244B68
:1017C8001A6000F03FFF0546204C04E000F03AFFA5
:1017D800401B022834D8236813F0007FF6D000207D
:1017E80031E000221A4B1A6000F02CFF0546174C16
:1017F80004E000F027FF401B022823D8236813F0D9
:10180800007FF6D100201EE001201CE003201AE032
:10181800032018E0012016E0032014E0032012E062
:10182800032010E003200EE003200CE003200AE070
:10183800032008E0002006E0012004E0032002E085
:10184800032000E0032002B0BDE8F0810010024050
:101858006000424230B486B0164D02AC2868696810
:10186800AA68EB680FC42B8AADF80430124B5B688A
:1018780003F00C02082A19D1C3F3834206A90A44CB
:1018880012F8102C13F4803F0CD00B4B5B68C3F399
:1018980040430B4413F8143C0848B0FBF3F002FB38
:1018A80000F004E0064800FB02F000E0034806B040
:1018B80030BC7047785D00080010024000127A00C2
:1018C80000093D002DE9F04104460D46614B1B68B7
:1018D80003F007038B420BD25E4B1A6822F0070213
:1018E8000A431A601B6803F007038B4240F0998093
:1018F800236813F0020F06D0574B596821F0F00106
:10190800A2680A435A60236813F0010F50D0636835
:10191800012B05D1504A126812F4003F0DD183E023
:10192800022B05D14C4A126812F0007F05D17EE0E7
:10193800494A126812F0020F7CD0474A516821F0D8
:1019480003010B43536000F07DFE06466368012BDC
:101958000FD105E000F076FE801B404503D96CE00E
:101968003D4F41F288387B6803F00C03042BF1D11A
:101978001EE0022B15D105E000F064FE801B4045F7
:1019880003D95DE0344F41F288387B6803F00C03DB
:10199800082BF1D10CE000F055FE801B404503D91F
:1019A80051E02D4F41F288387B6813F00C0FF2D1CB
:1019B800284B1B6803F00703AB420AD9254B1A686A
:1019C80022F007022A431A601B6803F00703AB42A0
:1019D8003CD1236813F0040F06D01F4B596821F43B
:1019E800E061E2680A435A60236813F0080F07D0E1
:1019F800194B5A6822F46052216942EAC1025A60BE
:101A0800FFF728FF144B5B68C3F30313134AD35C37
:101A1800D840134A1060002000F0E4FD0020BDE823
:101A2800F0810120BDE8F0810120BDE8F0810120AE
:101A3800BDE8F0810120BDE8F0810320BDE8F08118
:101A48000320BDE8F0810320BDE8F0810120BDE856
:101A5800F08100BF00200240001002408C5D0008A9
:101A680000000020014B1868704700BF00000020EC
:101A780008B5FFF7F7FF044B5B68C3F30223034A7B
:101A8800D35CD84008BD00BF001002409C5D000830
:101A980030B4036A23F001030362026A436885696C
:101AA80025F073050C68254322F002028C68224356
:101AB800104CA04203D004F50064A04205D122F0E6
:101AC8000802CC68224322F004020A4CA04203D048
:101AD80004F50064A04205D123F440734C69234304
:101AE8008C692343436085614B684363026230BC61
:101AF800704700BF002C014030B4036A23F48073A0
:101B08000362026A4368C56925F073050C682543BA
:101B180022F400728C6842EA0422124CA04203D0DC
:101B280004F50064A04206D122F40062CC6842EABF
:101B3800042222F480620B4CA04203D004F5006416
:101B4800A04207D123F440534C6943EA04138C693B
:101B580043EA04134360C5614B68C363026230BC47
:101B6800704700BF002C014030B4036A23F480534F
:101B78000362056A4368C26922F4E6420C6842EAD5
:101B8800042425F400558A6845EA0232094DA84222
:101B980003D005F50065A84204D123F480434D69BC
:101BA80043EA85134360C4614B680364026230BC36
:101BB800704700BF002C014010B4036A046A24F087
:101BC80001040462846924F0F00444EA021223F058
:101BD8000A031943826101625DF8044B704700BF34
:101BE80010B4036A23F0100303628469036A24F4BF
:101BF800704444EA023223F0A00343EA01118261EF
:101C080001625DF8044B704710B4846824F47F4483
:101C180042EA032319430C4384605DF8044B704780
:101C280010B50B460268946824F070044968214393
:101C380021F007041968214391605A68502A1FD07F
:101C480002D8402A0BD010BD602A1FD0702A22D19A
:101C58000068D9689A681B69FFF7D6FF10BD02684B
:101C6800116A146A24F0010414620268946924F069
:101C7800F0041B6944EA031393610368196210BDF9
:101C8800006899681A69FFF797FF10BD006899689E
:101C98001A69FFF7A5FF10BD704700BF38B50446A5
:101CA80090F83C30012B17D0012580F83C500223D6
:101CB80080F83D30FFF7B4FF2368DA6822F040026D
:101CC800DA602368DA6822F48042DA6084F83D50EA
:101CD800002084F83C0038BD022038BD0368244A3F
:101CE800904212D002F5006290420ED0B0F1804FBF
:101CF8000BD0A2F59832904207D002F5806290424C
:101D080003D002F58062904203D123F070034A6841
:101D18001343174A904212D002F5006290420ED047
:101D2800B0F1804F0BD0A2F59832904207D002F55F
:101D38008062904203D002F58062904203D123F47E
:101D48004073CA68134323F080034A691A43026048
:101D58008B68C3620B688362054B984203D003F516
:101D68000063984201D10B69036301234361704703
:101D7800002C014010B50446B0B190F83D3013F086
:101D8800FF0F04D1002380F83C30FFF785FF0223C2
:101D980084F83D30214651F8040BFFF79FFF0123DB
:101DA80084F83D30002010BD012010BD30B4036A16
:101DB80023F010030362026A4368856925F4E64547
:101DC8000C6845EA042522F020028C6842EA0412D5
:101DD800114CA04203D004F50064A04206D122F0C1
:101DE8008002CC6842EA041222F040020A4CA04267
:101DF80003D004F50064A04207D123F440634C6982
:101E080043EA84038C6943EA8403436085614B6831
:101E18008363026230BC7047002C014038B5044629
:101E28000D4690F83C30012B64D0012380F83C30FB
:101E3800022380F83D300C2A55D8DFE802F0075419
:101E480054541A5454542E54545441000068FFF703
:101E58001FFE23689A6942F008029A6123689A690A
:101E680022F004029A61236899692A690A439A61EF
:101E780039E00068FFF79AFF23689A6942F4006224
:101E88009A6123689A6922F480629A6123689A6940
:101E9800296942EA01229A6125E00068FFF72CFED1
:101EA8002368DA6942F00802DA612368DA6922F005
:101EB8000402DA612368D9692A690A43DA6112E0FF
:101EC8000068FFF751FE2368DA6942F40062DA61BC
:101ED8002368DA6922F48062DA612368DA69296999
:101EE80042EA0122DA61012384F83D30002084F8B7
:101EF8003C0038BD022038BD10B401238B40046A71
:101F080024EA03030362036A8A40134303625DF809
:101F1800044B704710B5044600680122FFF7ECFF38
:101F280023680C4A934205D002F50062934203D11C
:101F3800012202E0012200E000221AB15A6C42F4A8
:101F480000425A6423681A6842F001021A600020AD
:101F580010BD00BF002C014010B404238B40046A5C
:101F680024EA03030362036A8A40134303625DF8A9
:101F7800044B704710B5044600680422FFF7ECFFD5
:101F880023685A6C42F400425A6423681A6842F083
:101F980001021A60002010BD90F83C30012B22D0BD
:101FA800012380F83C30CB6823F440728B681343DC
:101FB80023F480624B681A4322F400620B681A43C8
:101FC80022F480520B691A4322F400524B691A43D7
:101FD800896922F440420A4303685A64002380F85E
:101FE8003C30184670470220704700BF30B490F864
:101FF8003C30012B20D0012380F83C30022280F8AD
:102008003D200268546824F07004546002685568E2
:102018000C682C4354600268946824F0800494602F
:102028000268946849682143916080F83D30002334
:1020380080F83C30184600E0022030BC704700BFF2
:1020480010B490F82430012B21D0012380F82430DB
:1020580003689A6812F0010F0FD10F4A926812F0C4
:10206800010F0AD10D4A934207D15C6824F4702409
:102078000A6822435A60002304E0836A43F020037D
:1020880083620123002280F82420184600E0022001
:102098005DF8044B704700BF002801400024014050
:1020A80000F00700064AD36823F4E0631B041B0C06
:1020B80043EA002343F0BF6343F40033D36070471F
:1020C80000ED00E030B4164BDB68C3F30223C3F124
:1020D8000705042D28BF04251C1D062C01D9033B28
:1020E80000E00023012404FA05F5013D2940994048
:1020F80004FA03F3013B1A400A43002806DA00F009
:102108000F001201D2B2074B1A5407E01201D2B2E3
:1021180000F1604000F5614080F8002330BC704752
:1021280000ED00E014ED00E0420900F01F0001237B
:1021380003FA00F0014B43F82200704700E100E089
:102148000138B0F1807F0AD2064B5860F021064A68
:1021580082F823100020986007221A607047012037
:10216800704700BF10E000E000ED00E0042805D152
:10217800054B1A6842F004021A607047024B1A684D
:1021880022F004021A60704710E000E0704700BFB8
:1021980008B5FFF7FBFF08BD0022064BDA61064BC6
:1021A8001A6942F004021A611A6942F040021A617F
:1021B800704700BFB8000020002002400022064BF4
:1021C800DA61064B1A6942F002021A6158611A690B
:1021D80042F040021A617047B80000200020024017
:1021E8002DE9F04105468846284B1B7E012B49D036
:1021F8000122264B1A760368022B13D14CF2503079
:10220800FFF778F8002834D10120FFF7C5FF4CF21A
:102218005030FFF76FF801461D4B1A6922F004028F
:102228001A6129E04CF25030FFF764F818BB4FF000
:10223800FF33C8F80030AC6801214CF25037144E17
:1022480010E02046FFF7BAFF3846FFF753F8336926
:1022580023F002033361014610B1C8F800400BE0D7
:1022680004F50064EA68AB6803EBC223A342E8D82C
:1022780002E0012100E001210022044B1A76084601
:10228800BDE8F0810220BDE8F08100BFB800002061
:10229800002002402DE9F00F82B000252B46784F30
:1022A800DFF8E4C1DFF8E481764C8146E1E00126FD
:1022B8009E400A683240B24240F0DA8048681228EC
:1022C8002FD00BD8022829D003D868B3012820D0F2
:1022D80039E0032834D011281DD034E0DFF8B0A14C
:1022E800504521D008D8AAF5801A50451CD00AF5C7
:1022F800803A504527D117E0DFF898A1504513D010
:102308000AF5803A50450FD0AAF5801A50451AD1DF
:102318000AE0CD6817E0CD68043514E0CD680835CB
:1023280011E0CD680C350EE0886858B1012803D15A
:10233800C9F81060082506E0C9F81460082502E00D
:10234800002500E00425FF2A01D8484601E009F1EC
:102358000400FF2A01D89E0002E0A3F10806B60097
:10236800D0F800B04FF00F0A0AFA06FA2BEA0A0A68
:1023780005FA06F64AEA06060660486810F0805F25
:1023880076D0B86940F00100B861B86900F0010082
:10239800019001989808861C5CF826B003F00306A3
:1023A800B6004FF00F0A0AFA06FA2BEA0A0AC145E4
:1023B80025D0DFF8E4B0D9451ED00BF5806BD945A0
:1023C80017D00BF5806BD94510D00BF5806BD9452C
:1023D80009D00BF5806BD94502D14FF0050B10E001
:1023E8004FF0060B0DE04FF0040B0AE04FF0030B23
:1023F80007E04FF0020B04E04FF0010B01E04FF053
:10240800000B0BFA06F646EA0A0602304CF8206082
:10241800486810F4803F03D020681043206003E030
:10242800206820EA02002060486810F4003F03D0CA
:1024380060681043606003E0606820EA0200606042
:10244800486810F4801F03D0A0681043A06003E020
:10245800A06820EA0200A060486810F4001F03D0BA
:10246800E0680243E26003E0E06820EA0202E2601A
:1024780001330F2B7FF61BAF02B0BDE8F00F70479A
:102488000010024000040140000001400008014023
:102498000000211000003110000C014083680B423D
:1024A80001D0012070470020704700BF0AB10161C8
:1024B8007047090401617047C3685940C16070479B
:1024C8002DE9F04182B00446036813F0010F60D093
:1024D800404BDB6913F0805F0BD13E4BDA6942F069
:1024E8008052DA61DB6903F080530193019B012775
:1024F80000E00027384B1B6813F4807F12D1364B5D
:102508001A6842F480721A6000F09CF80646324D50
:1025180004E000F097F8801B642852D82B6813F465
:10252800807FF6D02B4B1B6A13F4407325D062686A
:1025380002F440729A4220D0264A136A23F440706B
:10254800264901250D6000250D60106213F0010F6A
:1025580013D000F077F8804605F1804505F504357D
:1025680041F2883605E000F06DF8C8EB0000B04293
:1025780029D82B6A13F0020FF5D0164B196A21F4EB
:10258800407162680A431A621FB1DA6922F0805208
:10259800DA61236813F0020F06D00E4B596821F454
:1025A8004041A2680A435A60236813F0100F0CD008
:1025B800084B5A6822F4800261690A435A60002075
:1025C80004E0032002E0032000E0002002B0BDE8A0
:1025D800F08100BF001002400070004040044242F9
:1025E800704700BF10B50446074B1868074BA3FB9C
:1025F80000208009FFF7A4FD4FF0FF30214600229C
:10260800FFF760FD002010BD00000020D34D6210D0
:1026180008B5074B1A6842F010021A600320FFF74A
:102628003FFD0020FFF7DEFFFFF7DAFF002008BDBF
:1026380000200240024B1A6801321A60704700BF3E
:10264800D8000020014B1868704700BFD800002050
:1026580030B583B00190FFF7F5FF0546019CB4F152
:10266800FF3F00D00134FFF7EDFF401BA042FAD333
:1026780003B030BD704700BF30B482B0002301936F
:1026880090F82430012B00F08980012380F8243051
:102698004B68062B0ED80268546B03EB8303053B8B
:1026A8001F259D4024EA05050C6804FA03F32B4313
:1026B80053631EE00C2B0ED80268146B03EB8303E4
:1026C800233B1F259D4024EA05050C6804FA03F303
:1026D8002B4313630DE00268D46A03EB8303413B89
:1026E8001F259D4024EA05050C6804FA03F32B43D3
:1026F800D3620B68092B0ED90268D46803EB430335
:102708001E3B07259D4024EA05058C6804FA03F35F
:102718002B43D3600CE00268146903EB43030725DD
:102728009D4024EA05058C6804FA03F32B431361E2
:102738000B68103B012B27D803681A4A93421DD116
:102748009A6812F4000F21D19A6842F400029A6044
:102758000B68102B1CD1144B1A68144BA3FB0213E3
:102768009B0C03EB83035B00019302E0019B013B9D
:102778000193019B002BF9D100220AE0836A43F000
:1027880020038362012204E0002202E0002200E02C
:102798000022002380F82430104600E0022002B016
:1027A80030BC7047002401400000002083DE1B433A
:1027B80030B583B004460023019303689A6812F089
:1027C800010F2ED19A6842F001029A60164B1A68DE
:1027D800164BA3FB02139B0C019302E0019B013BE8
:1027E8000193019B002BF9D1FFF72CFF054611E05F
:1027F800FFF728FF401B02280CD9A36A43F01003F7
:10280800A362E36A43F00103E362002384F82430FF
:10281800012007E023689B6813F0010FE8D000202F
:1028280000E0002003B030BD0000002083DE1B4321
:1028380010B5044690F82430012B6ED0012380F89F
:102848002430FFF7B5FF0246002861D1A36A23F4BC
:10285800407323F0010343F48073A3622368304973
:102868008B4205D1A1F58061496811F4702F0ED112
:10287800A16A21F48011A162596811F4806F1CD0FB
:10288800A16A21F4405141F48051A16215E0A16A86
:1028980041F48011A16223498B4203D001F5806184
:1028A8008B420AD11F49496811F4806F05D0A16A8B
:1028B80021F4405141F48051A162A16A11F4805F72
:1028C80004D0E16A21F00601E16201E00021E16241
:1028D800002184F824106FF00201196023689968B8
:1028E80001F46021B1F5602F0DD10D498B4205D15E
:1028F800A1F58061496811F4702F04D1996841F4F9
:10290800A001996007E0996841F48011996002E09C
:10291800002384F82430104610BD022010BD00BFEB
:10292800002801400024014038B5044603689A682D
:1029380012F0010F1DD09A6822F001029A60FFF789
:1029480081FE05460EE0FFF77DFE401B022809D9EF
:10295800A36A43F01003A362E36A43F00103E3624E
:10296800012038BD23689B6813F0010FEBD10020CC
:1029780038BD002038BD00BF70B50446002800F0FF
:102988008680836A23B9C36280F82430FFF772FE19
:102998002046FFF7C9FFA36A13F0100F71D1002872
:1029A8006FD1A36A23F4885323F0020343F0020390
:1029B800A36261682368374A934206D1E269B2F597
:1029C800402F03D14FF4002200E0E2690A43E56892
:1029D80042EA4502A168B1F5807F04D0012905D1FA
:1029E8004FF4807103E04FF4807100E000216669C4
:1029F800012E0FD135B9A569013D41EA453141F4B0
:102A0800006107E0A56A45F02005A562E56A45F082
:102A18000105E5625D6825F4694529435960216827
:102A28008D681D4B2B4013438B60A368B3F5807FE3
:102A380001D0012B03D12569013D2D0500E00025BA
:102A48002368D96A21F470012943D96223689968F7
:102A5800124B0B409A4208D10023E362A36A23F089
:102A6800030343F00103A36270BDA36A23F01203BA
:102A780043F01003A362E36A43F00103E362012019
:102A880070BDA36A43F01003A362012070BD01204A
:102A980070BD00BF003C0140FDF7E1FFFE0E1FFFC7
:102AA80003685A6912F4806F0DD06FF480625A611E
:102AB8000423036400230363202280F83D2080F868
:102AC8003C30012070470020704700BF2DE9F843D3
:102AD80007460D4691461E46C1F3074815E0B6F174
:102AE800FF3F12D02EB1FFF7ADFD089BC01AB042D0
:102AF8000BD900233B63202287F83D2087F83E301E
:102B080087F83C300320BDE8F883B8F1010F09D1FC
:102B18003B685C6925EA0404A4B2D4F1010438BF17
:102B2800002408E03C68A46925EA0404A4B2D4F1AE
:102B3800010438BF00244C45D1D00020BDE8F883FB
:102B48002DE9F84304460E4690469946C1F30747D7
:102B58002EE02068456915F4806F13D0036843F4AC
:102B68000073036023686FF480625A61042323644E
:102B780000232363202284F83D2084F83C30012080
:102B8800BDE8F883B8F1FF3F12D0B8F1000F05D0C7
:102B9800FFF758FDC9EB0000404509D9002323631E
:102BA800202284F83D2084F83C300320BDE8F883D7
:102BB800012F08D12368586926EA000080B2003046
:102BC80018BF012007E02368986926EA000080B250
:102BD800003018BF01200028BBD1BDE8F88300BF32
:102BE800F0B583B004460F4616461D46C06A042851
:102BF80004D0012802D010F5803F05D123681A6857
:102C080042F480721A6007E0236B122B04D1236808
:102C18001A6842F480721A60009520464FF001113C
:102C280000223346FFF752FF58BB2369B3F5804FA4
:102C380004D1236807F0FE071F6115E0236807F435
:102C48004072D21142F0F0021A6120461149324610
:102C58002B46FFF775FF20B1236C042B13D10123FA
:102C680014E02368FFB21F6120460B4932462B4609
:102C7800FFF766FF034648B1236C042B05D10123F7
:102C880004E0032302E0032300E00323184603B013
:102C9800F0BD00BF08000100020001002DE9F0416D
:102CA80084B00446884617461E46C06A25682B68C5
:102CB80043F480632B60042804D0012802D010F567
:102CC800803F05D123681A6842F480721A6007E0D1
:102CD800236B112B04D123681A6842F480721A609E
:102CE800009620464FF0011100223B46FFF7EEFE0A
:102CF800002852D12369B3F5804F06D1236848F0E4
:102D080001085FFA88F21A613AE0236808F440750E
:102D1800ED0945F0F0021A61204626493A46334645
:102D2800FFF70EFF20B1236C042B38D101233DE0BF
:102D380023685FFA88F21A6120461F493A463346EB
:102D4800FFF7FEFE20B1236C042B2AD101232DE0CE
:102D580000220392236859690391996903910399A1
:102D6800196841F480711960009620464FF00111EE
:102D78003B46FFF7ABFEB0B9236845F0F1051D618E
:102D880020460D493A463346FFF7DAFE034668B156
:102D9800236C042B09D1012308E0032306E0032355
:102DA80004E0032302E0032300E00323184604B0F1
:102DB800BDE8F081080001000200010070B504467A
:102DC8000D46164619E02046FFF76AFEE0B9B5F150
:102DD800FF3F12D025B1FFF735FC801BA8420CD964
:102DE800236C43F02003236400232363202284F808
:102DF8003D2084F83C30032070BD23685B6913F0E4
:102E0800800FE0D0002070BD012070BD70B5044671
:102E18000D46164619E02046FFF742FEE0B9B5F127
:102E2800FF3F12D025B1FFF70DFC801BA8420CD93B
:102E3800236C43F02003236400232363202284F8B7
:102E48003D2084F83C30032070BD23685B6913F093
:102E5800040FE0D0002070BD012070BDF8B5064613
:102E68000D46174622E0596911F0100F0CD06FF08B
:102E780010025A61002333643363202286F83D2010
:102E880086F83C300120F8BD25B1FFF7DBFBC01BFD
:102E9800A8420BD9336C43F020033364202386F80F
:102EA8003D30002386F83C300320F8BD33685C6968
:102EB80014F0400FD7D00020F8BD00BF704700BF06
:102EC80038B50446002800F0838090F83D3013F0B0
:102ED800FF0F04D1002380F83C30FFF7EFFF2423D5
:102EE80084F83D3023681A6822F001021A60FEF760
:102EF800BFFD384BA3FB00239B0C2268536021685D
:102F08006268354DAA4201D8013308E04FF4967241
:102F180002FB03F3314AA2FB03539B0901330B6203
:102F2800226863682C498B4208D85B00B0FBF3F039
:102F3800C0F30B03032B2DD804202BE0A16851B953
:102F480003EB4305B0FBF5F5C5F30B05D5F101051A
:102F580038BF00250BE003EB830505EB8505B0FBC7
:102F6800F5F5C5F30B05D5F1010538BF002585B981
:102F780031B903EB4303B0FBF3F040F4004009E040
:102F880003EB830303EB8303B0FBF3F040F440400F
:102F980000E00120D0612368E169226A0A431A60CF
:102FA80023682169E2680A439A6023686169A26913
:102FB8000A43DA6023681A6842F001021A600020A6
:102FC8002064202384F83D30206384F83E0038BD17
:102FD800012038BD83DE1B43A0860100D34D62105B
:102FE8002DE9F04385B004460F4691469846FFF711
:102FF80029FB064694F83D50EDB2202D40F0A08004
:1030080000902046554901221923FFF75FFD00284B
:1030180040F0988094F83C30012B00F09580012313
:1030280084F83C3023681A6812F0010F03D11A683B
:1030380042F001021A6023681A6822F400621A60DA
:10304800212384F83D30102384F83E300023236484
:10305800C4F82490A4F82A80A3F58033E362638D32
:103068002385204639460C9A3346FFF7B9FD0546B5
:1030780060B1236C042B04D1002384F83C30012573
:1030880067E0002384F83C30032562E000230393C3
:1030980023685A6903929B690393039B3FE0204688
:1030A8000C993246FFF78AFE48B1236C042B4DD1A8
:1030B80023681A6842F400721A60012549E0226800
:1030C800636A591C61621B781361638D013B9BB273
:1030D8006385238D013B9BB223852268516911F0DA
:1030E800040F0CD05BB1636A591C61621B781361D1
:1030F800638D013B9BB26385238D013B238520466D
:103108000C993246FFF782FE48B1236C042B1FD17D
:1031180023681A6842F400721A60012519E0238DA9
:10312800002BBCD123681A6842F400721A6020236D
:1031380084F83D30002384F83E3084F83C3008E0C1
:10314800022506E0022504E0022502E0032500E04E
:103158000325284605B0BDE8F08300BF0200100033
:103168002DE9F04387B004460F4691469846FFF78D
:1031780069FA064694F83D50EDB2202D40F05F8183
:1031880000902046954901221923FFF79FFC00284B
:1031980040F0578194F83C30012B00F05481012312
:1031A80084F83C3023681A6812F0010F03D11A68BA
:1031B80042F001021A6023681A6822F400621A6059
:1031C800222384F83D30102384F83E300023236402
:1031D800C4F82490A4F82A80A3F58033E362638DB1
:1031E8002385204639460E9A3346FFF757FD054694
:1031F80060B1236C042B04D1002384F83C300125F2
:103208002CE1002384F83C30032527E1238D5BB9AA
:10321800029323685A6902929A690292029A1A687A
:1032280042F400721A60FAE0012B13D123681A687D
:1032380022F480621A6072B60023039323685A69E5
:1032480003929A690392039A1A6842F400721A6008
:1032580062B6E4E0022B13D123681A6842F40062D4
:103268001A6072B60023049323685A6904929A6913
:103278000492049A1A6822F480621A6062B6CEE058
:1032880023681A6842F480621A6000230593236851
:103298005A6905929B690593059BC0E0032B00F2D0
:1032A8009180012B19D120460E993246FFF7D6FDA1
:1032B80028B1236C202B40F0C8800325CEE0636A38
:1032C8005A1C6262226812691A70238D013B238599
:1032D800638D013B9BB26385A4E0022B2BD1009642
:1032E800204641463A460E9BFFF7F0FB002840F087
:1032F800AE8072B623681A6842F400721A60636A74
:103308005A1C6262226812691A70238D013B238558
:10331800638D013B9BB2638562B6636A5A1C626225
:10332800226812691A70238D013B2385638D013B46
:103338009BB2638576E00096204641463A460E9B4E
:10334800FFF7C4FB002840F0848023681A6822F441
:1033580080621A6072B6636A5A1C626222681269D5
:103368001A70238D013B2385638D013B9BB26385D6
:103378000096204641463A460E9BFFF7A7FB0028D9
:1033880069D123681A6842F400721A60636A5A1C89
:103398006262226812691A70238D013B2385638D4E
:1033A800013B9BB2638562B6636A5A1C62622268FB
:1033B80012691A70238D013B2385638D013B9BB2F3
:1033C80063852FE020460E993246FFF747FD38B156
:1033D800236C202B41D1032540E000BF02001000E0
:1033E800636A5A1C6262226812691A70238D013B53
:1033F8002385638D013B9BB2638523685A6912F06C
:10340800040F0FD0626A511C61621B691370238D0F
:10341800013B2385638D013B9BB2638502E0DFF8A6
:1034280044800027238D002B7FF438AF202384F8B5
:103438003D30002384F83E3084F83C300EE002250D
:103448000CE002250AE0022508E0012506E0032534
:1034580004E0032502E0032500E00125284607B023
:10346800BDE8F0830400010010B4034600283CD0F6
:10347800026820498A420AD81F4911441F4AA2FB00
:1034880001010909890019641D4ADA6309E01D4927
:1034980011441A4AA2FB01010909890019641A4A50
:1034A800DA63022283F8212019680A6822F47F521D
:1034B80022F030025C6898680443D86804431869AD
:1034C80004435869044398690443D8692043024374
:1034D8000A6000209862D8621863586398630122D2
:1034E80083F8212083F8200000E001205DF8044BD8
:1034F800704700BF07040240F8FFFDBFCDCCCCCC1D
:1035080000000240F8FBFDBF000402400F4B1A68A0
:1035180042F001021A6059680D4A0A405A601A6856
:1035280022F0847222F480321A601A6822F480220F
:103538001A605A6822F4FE025A604FF41F029A6019
:103548004FF00062034B9A60704700BF00100240C2
:103558000000FFF800ED00E02DE9F0418AB04A4D87
:10356800EB6943F48003EB61EB6903F48003019397
:10357800019B6B6943F001036B616B6903F0010305
:103588000293029B0E2001210422FEF79BFD0E20D0
:10359800FEF7CAFD0F2001210322FEF793FD0F203D
:1035A800FEF7C2FD394E3A4B33603A4B7360002444
:1035B800B460F4604FF4804333617461B461F461C2
:1035C80034623046FFF77CFC6B6943F001036B61A2
:1035D8006B6903F001030393039BAB6943F0080392
:1035E800AB61AB6903F008030493049B4FF4406399
:1035F800069312230793012308930323099326486C
:1036080006A9FEF747FEEB6943F48003EB61EB691B
:1036180003F480030593059B204D214B2B606C60C0
:10362800AC604FF08008C5F80C802C616C61AC610F
:103638004FF48057EF612846FFF716FFB5636E62B7
:10364800184D194B2B6010236B60AC60C5F80C80CB
:103658002C616C61AC61EF612846FFF705FF75636B
:103668006E62212021462246FEF72CFD2120FEF71E
:103678005BFD222021462246FEF724FD2220FEF78C
:1036880053FD0AB0BDE8F08100100240500100204F
:1036980000580040400D0300000C0140E4010020E8
:1036A8005800024028020020440002402DE9F04F53
:1036B80089B0814B9A6942F004029A619A6902F0D2
:1036C80004020192019A9A6942F008029A619A6981
:1036D80002F008020292029A9A6942F010029A6174
:1036E8009B6903F010030393039B00230593069340
:1036F8004FF00208CDF81C804FF0200A0DEB0A04A9
:1037080044F810AD6D4F38462146FEF7C3FD4023FF
:10371800049338462146FEF7BDFD4FF0800BCDF8E7
:1037280010B038462146FEF7B5FD4FF48063049388
:10373800634D28462146FEF7ADFD4FF40063049320
:1037480028462146FEF7A6FD4FF4805604962846E3
:103758002146FEF79FFD049606F1804606F5784659
:1037680030462146FEF796FDCDF8108030462146BA
:10377800FEF790FD4FF00109CDF81490042304934F
:1037880038462146FEF786FD10230493304621462D
:10379800FEF780FDCDF810A030462146FEF77AFDF1
:1037A80003230593CDF8109028462146FEF772FDB5
:1037B800CDF8109030462146FEF76CFD082304939F
:1037C80028462146FEF766FDCDF81080284621469A
:1037D800FEF760FD1023049328462146FEF75AFDA4
:1037E800CDF810A028462146FEF754FD0423049383
:1037F80028462146FEF74EFD08230493304621460D
:10380800FEF748FD0423049330462146FEF742FDA7
:10381800CDF814804023049328462146FEF73AFD4C
:10382800CDF810B028462146FEF734FD4FF4807AD3
:10383800CDF810A028462146FEF72CFDCDF810B093
:1038480030462146FEF726FDCDF810903846214631
:10385800FEF720FDCDF8108038462146FEF71AFD08
:10386800CDF810A030462146FEF714FD4FF4007342
:10387800049330462146FEF70DFD4FF48063049310
:1038880030462146FEF706FD4FF4005304933846B0
:103898002146FEF7FFFC4FF4804304933846214647
:1038A800FEF7F8FC4FF40043049338462146FEF730
:1038B800F1FC09B0BDE8F08F00100240000C014097
:1038C800001001402DE9F04F99B0754B9A6942F408
:1038D80000629A619A6902F400620192019A9A69F7
:1038E80042F400529A619B6903F400530293029BCD
:1038F8006C4EDFF8B891C6F80090002474604FF061
:103908002008C6F808804FF4FA6BC6F80CB034618A
:103918007461B4613046FEF72DFA1023169317949C
:10392800304616A9FEF762FB60230F93109411949A
:1039380008271297139414944FF400731593304684
:103948000FA92246FEF76AFA30460FA90422FEF7AD
:1039580065FA30460FA93A46FEF760FA4FF400635D
:1039680008934FF4806309930A94CDF82C800C9443
:103978000D940E9430460DEB0801FEF70DFB4A4DF1
:10398800DFF82CA1C5F800A06C60C5F80880C5F860
:103998000CB02C616C61AC612846FEF7EBF9CDF8F0
:1039A800588080231793284616A9FEF71FFB049416
:1039B80018A9052341F8543D2846FEF76FF96023FE
:1039C8000F93109411941297139414944FF4007356
:1039D800159328460FA92246FEF720FA28460FA974
:1039E8000422FEF71BFA28460FA93A46FEF716FAF4
:1039F8004FF4006308934FF4806309930A94CDF859
:103A08002C800C940D940E9428460DEB0801FEF7BB
:103A1800C3FADAF8443023F40043CAF84430D9F83A
:103A2800443023F40043C9F8443028462146FEF7C1
:103A380071FA28460421FEF76DFA28463946FEF742
:103A480069FA28462146FEF795FA28460421FEF72A
:103A580091FA28463946FEF78DFA30462146FEF798
:103A680059FA30460421FEF755FA30463946FEF732
:103A780051FA30462146FEF77DFA30460421FEF71A
:103A880079FA30463946FEF775FA2B6801221A632F
:103A980033681A6842F001021A6019B0BDE8F08F65
:103AA80000100240A401002034030020002C014033
:103AB800003401402DE9F04186B0424EB36943F429
:103AC8000073B361B36903F400730093009B3E4C29
:103AD8003E4B23604FF48073A3600025E560656169
:103AE8004FF44023E36165604FF00508C4F8108087
:103AF8002046FEF741FF364B5A6842F480225A604E
:103B080006A94FF4C02341F8043D2046FEF798FA71
:103B1800012304930E2202920393204602A9FEF782
:103B2800ABFD029502270397204602A9FEF7A4FDE4
:103B380004970B27029703230393204602A9FEF755
:103B48009BFD0C23029304230393204602A9FEF74E
:103B580093FD0723049310230293CDF80C8020468D
:103B680002A9FEF789FD23689A6842F4000242F42C
:103B780080729A609A6842F001029A60736943F011
:103B880001037361736903F001030193019B114BF6
:103B98001D60C3F80480104A9A60104ADA6040F643
:103BA800A2221A601A6842F001021A6038462946B1
:103BB8002A46FEF787FA3846FEF7B6FA06B0BDE899
:103BC800F08100BF001002406C0200200024014078
:103BD80000000140080002404C240140E00200209F
:103BE800F0B585B0284B9A6942F480629A619B6966
:103BF80003F480630093009B244C254B23604FF40F
:103C08008073A3600023E36063614FF46022E26184
:103C18006360052626612046FEF7AEFE0123039366
:103C28000F2201920293204601A9FEF725FD0D23DC
:103C3800019302250295204601A9FEF71DFD039573
:103C48000A23019303270297204601A9FEF714FDD2
:103C580001950423029320460DEB0301FEF70CFDAA
:103C68000723039301970296204601A9FEF704FD56
:103C780023689A6842F480729A609A6842F0010256
:103C88009A6005B0F0BD00BF00100240200100207E
:103C98000028014000B583B00A2300930648A421F8
:103CA800064A0123FFF75CFA08B9012000E000206A
:103CB80003B05DF804FB00BF500100206C00002039
:103CC80070B582B0104CF0232370552363700F4DEC
:103CD800642600962846A42122460223FFF780F98D
:103CE8000A20FEF7B5FCFB232370002363700096BF
:103CF8002846A42122460223FFF772F90A20FEF77C
:103D0800A7FC02B070BD00BFB40300205001002022
:103D180030B583B00F4A002313700F4C0A25009565
:103D28002046A4210123FFF75BF90320FEF790FC4E
:103D380000952046A421094A0623FFF711FA18B96D
:103D48000022074B1A6003E0054B1A6801321A601B
:103D580003B030BDB4030020500100206C000020E7
:103D68000400002070B50D4B1B681333262B14D8A4
:103D780000240B4B1C700B4B1C700B4E642504E08D
:103D880034702846FEF764FC0134072CF8DD074838
:103D980020210022FEF78AFBFEE770BD7404002094
:103DA80080000020940000209C00002000080140B2
:103DB80010B5054C052323704FF4FA70FEF748FC44
:103DC8000023237010BD00BF9C00002010B5044CD8
:103DD800052323706420FEF73BFC0023237010BDED
:103DE8009C00002008B5FDF767FA044B1888044BBF
:103DF800198801F063FCFDF773FA08BD080000207C
:103E08007400002030B597B002250C95012310935B
:103E1800102311931395002414944FF460131593F1
:103E28000CA8FDF70DFB0F230793089509944FF491
:103E380080630A930B9407A82946FDF743FD019573
:103E48004FF44043039301A8FEF73AFBFDF70AFE3F
:103E5800084BA3FB00208009FEF772F90420FEF747
:103E680085F94FF0FF3021462246FEF72BF917B0AF
:103E780030BD00BFD34D62102DE9F04F89B0FEF779
:103E8800C7FBA34CA36943F00103A361A36903F033
:103E980001030793079B0320FEF702F96FF00B005D
:103EA80000210A46FEF70EF96FF00A0000210A46C3
:103EB800FEF708F96FF0090000210A46FEF702F93B
:103EC8006FF0040000210A46FEF7FCF86FF00300CB
:103ED80000210A46FEF7F6F86FF0010000210A46B5
:103EE800FEF7F0F84FF0FF3000210A46FEF7EAF837
:103EF800FFF788FF636923F001036361FFF7D6FBCF
:103F0800FFF7E0FCFFF7D6FDFFF76AFE81482021A6
:103F18000122FEF7CBFA8048FEF78AFC7F48FEF7BD
:103F280087FC04247E4E642505E063003370284630
:103F3800FEF78EFB013C002CF7DA0424784E64254A
:103F480006E06300013B33702846FEF781FB013C25
:103F5800002CF6DA0022724B1A700122714B1A708B
:103F6800FDF7AAF901F012FA6F4C704B1888214638
:103F780001F0EAF9FDF7B4F92088FCF7ADFA002260
:103F88006B4BFCF739FCFCF7EFFD8346FCF7B6FA00
:103F98005DA3D3E90023FCF777FD08B14FF07E5B02
:103FA800FFF7DAFA634C272384F840300527676463
:103FB80004F148006049542201F0C4FE012626702D
:103FC800002584F83C50204601F09CFD3220FEF785
:103FD8003FFB204601F0DAFC3220FEF739FB204691
:103FE80029462A4601F0B2FC2046544901F0B8FCA3
:103FF80020462946324601F0A9FC2046504901F0E6
:10400800AFFC204601F0C2FC3846FEF721FB2046F3
:104018002946324601F09AFC20464A4901F0A0FCA4
:1040280020460821324601F091FC2046464901F01D
:1040380097FC20460F21324601F088FC2046434970
:1040480001F08EFC204629462A4601F07FFC2046D6
:104058003F4901F085FC204608212A4601F076FCFC
:1040680020463C4901F07CFC20460E212A4601F0FE
:104078006DFC2046384901F073FC3848042132466B
:10408800FEF714FA364B1B8A264B1E700295AA4679
:104098000220FEF7DDFA1F480221FEF7FFF900288B
:1040A8007AD000221F4B1A701A4D02240A2602E009
:1040B8003046FEF7CDFA28462146FEF7EFF90028EC
:1040C800F6D1FFF783FE4FF49670FEF7C1FA114858
:1040D8000221FEF7E3F920B944E03046FEF7B8FACA
:1040E80002E00C4D02240A2628462146FEF7D6F99E
:1040F8000028F2D1FFF75CFE4FF4AF70FEF7A8FA84
:10410800FFF730FE48E000BF9A9999999999C93FFD
:1041180000100240000801406C020020200100202D
:104128009C0000209400002074000020080000205B
:1041380000408F40B803002050010020A45D000813
:10414800B85D0008C85D0008D05D0008D45D0008AF
:10415800D85D0008E05D0008E45D0008000C01403F
:10416800E002002058464FF07A51FCF753FD834691
:10417800FCF7C4F99CA3D3E90023FCF7A3FC08B11E
:104188004FF07C5B5846A249FCF74CFEFDF736F829
:10419800A04B1880FFF726FE9F4B5B8A9BB2B43B6F
:1041A800B3F5805F0BDA9C4B5B8A9BB2B42B04D4CB
:1041B800994B5E8AB43EB6B203E0002601E040F6B1
:1041C800FF76954BD88980B2A0F50060FCF784F99A
:1041D80000224FF07D53FCF7E5F9FCF7C5FC0746D4
:1041E8008E4B1860039658468D49FCF71BFEFCF76A
:1041F800DFFF361A8B4B1E608B4B1B78002B40F071
:10420800DE815046FCF7BAFD8849FCF70BFEFCF747
:1042180075F9804689463046FCF75EF904460D4636
:1042280000220023FCF730FC28B17342322BD4BFA4
:104238000023012303E0322ED4BF0023012373B1EE
:104248002046294600220023FCF71EFC18B17042C4
:10425800FCF794FD04E03046FCF790FD00E074485C
:104268003946FCF7DFFDFCF749F961A3D3E90023E0
:10427800FCF798F902460B4620462946FBF7E0FF73
:1042880000226C4BFCF71EFC002876D120462946FC
:1042980000220023FCF7F8FB28B17342322BD4BF6D
:1042A8000023012303E0322ED4BF0023012373B17E
:1042B8002046294600220023FCF7E6FB18B170428D
:1042C800FCF75CFD04E03046FCF758FD00E0584878
:1042D8003946FCF7A7FDFCF711F945A3D3E90023FC
:1042E800FCF760F902460B4620462946FBF7A8FF73
:1042F80041A3D3E90023FCF7C7FB002837D12046A8
:10430800294600220023FCF7BFFB28B17342322B59
:10431800D4BF0023012303E0322ED4BF002301239E
:1043280073B12046294600220023FCF7ADFB18B1E3
:104338007042FCF723FD04E03046FCF71FFD00E067
:104348003B483946FCF76EFDFCF7D8F828A3D3E9BB
:104358000023FCF727F902460B4620462946FBF7BF
:104368006FFF27A3D3E90023FCF71CF902E04FF005
:10437800AA60314902460B4602E023A3D3E9002391
:1043880040464946FBF75CFFFCF7A6FB80460298CF
:10439800FCF7F4FC2549FCF745FDFCF7AFF8CDE93F
:1043A80004012046294600220023FCF76DFB28B1B2
:1043B8007342322BD4BF0023012303E0322ED4BF33
:1043C80000230123D3B32046294600220023FCF70B
:1043D8005BFB18B17042FCF7D1FC30E03046FCF7CB
:1043E800CDFC2CE0AFF30080CDCCCCCCCCCC0440C1
:1043F800333333333333F3BF0000000000908AC0F7
:10440800000000A09999C9BF00005005004065C090
:1044180000007A4474000020E0020020800400209C
:104428000020A8447C04002076000020CDCC4C3F1E
:104438000000484200908A4000406540764839466E
:10444800FCF7F0FCFCF75AF84FF03332734BFCF7EB
:10445800A9F802460B4620462946FBF7F1FE002242
:104468006F4BFCF72FFB002876D120462946002207
:104478000023FCF709FB28B17342322BD4BF002379
:10448800012303E0322ED4BF0023012373B1204659
:10449800294600220023FCF7F7FA18B17042FCF70E
:1044A8006DFC04E03046FCF769FC00E05A483946E8
:1044B800FCF7B8FCFCF722F84FF03332574BFCF707
:1044C80071F802460B4620462946FBF7B9FE4CA375
:1044D800D3E90023FCF7D8FA002837D1204629462B
:1044E80000220023FCF7D0FA28B17342322BD4BF44
:1044F8000023012303E0322ED4BF0023012373B12C
:104508002046294600220023FCF7BEFA18B1704263
:10451800FCF734FC04E03046FCF730FC00E03E4891
:104528003946FCF77FFCFBF7E9FF4FF033323B4B92
:10453800FCF738F802460B4620462946FBF780FE72
:1045480031A3D3E90023FCF72DF802E04FF0AA606D
:10455800344902460B4602E02DA3D3E90023DDE9E6
:104568000401FBF76DFEFCF7B7FA0AF13203434585
:104578001FDDAAF1320AC2451BDA029901F13203A2
:10458800834216DDA1F13203834212DA002E02DDE6
:104598000122254B1A7016F5967F07DD4242234B00
:1045A8001A60C8F10002224B1A6002E000221E4B7A
:1045B8001A7000221F4B1A600290C2463DE1FFF7B5
:1045C800A7FB0122184B1A701B4B1B787F3BDB00A3
:1045D800B3F57A7F04DC194EB342A8BF1E4601E04A
:1045E8004FF47A76164B1E60134B5B78803BDB00EA
:1045F800B3F57A7F26DC114FBB42A8BF1F4623E0E4
:104608000000000000908AC0000000A09999C9BF6E
:1046180000005005004065C0000048423333F33FB6
:1046280000908A400040654094000020A0000020CF
:1046380098000020040000206C00002018FCFFFFF8
:10464800840400204FF47A775B4B1F60DFF8848185
:10465800D8F80000FBF740FF51A3D3E90023FBF78C
:10466800A1FF04460D463046FBF736FF4EA3D3E9BB
:104678000023FBF797FF02460B4620462946FBF727
:10468800DFFDFCF729FA0646C8F80000DFF8488184
:10469800D8F80000FBF720FF41A3D3E90023FBF77C
:1046A80081FF04460D463846FBF716FF3EA3D3E9C3
:1046B8000023FBF777FF02460B4620462946FBF707
:1046C800BFFDFCF709FAC8F80000FBF705FF34A3A3
:1046D800D3E90023FBF766FF804689463046FBF79F
:1046E800FBFE0022354BFBF75DFF04460D464046B6
:1046F800494622462B46FBF7A1FD06460F460022F7
:104708002F4BFCF7DFF978B93046394628A3D3E9AF
:104718000023FCF7B9F928B930463946FCF7DCF92B
:10472800064603E0274E01E04FF4617640464946CD
:1047380022462B46FBF784FD04460D460022204BFB
:10474800FCF7C0F978B92046294619A3D3E9002314
:10475800FCF79AF928B920462946FCF7BDF9044622
:1047680003E0184C01E04FF461740AF164039C42C1
:1047780034DAAAF1640A544530DD029A02F164037E
:104788009E422BDAA2F164039E4227DD0E4B1B6882
:10479800042B23D80D4B1E600D4B1C604BE000BF53
:1047A800CDCCCCCCCCCCEC3F9A9999999999B93F7E
:1047B8000000000000208CC0680400200000E03FDA
:1047C80000208C407CFCFFFF04000020A00000209B
:1047D800980000206C04002074040020964B1B688D
:1047E800052B28D90025954B1D60954B1D60954BD1
:1047F8001D70954F384629462A4601F0A7F83846D5
:10480800924901F0ADF8384608212A4601F09EF891
:1048180038468F4901F0A4F838460E212A4601F09F
:1048280095F838468B4901F09BF84FF47A70FDF7FC
:104838000FFF894B1D700296A2460398FBF74CFEAA
:104848007BA3D3E90023FBF7D7FF06460F4658465C
:10485800FBF754FE04460D463046394622462B46A1
:10486800FBF7ECFC00227D4BFCF72CF968B3002029
:10487800002122462B46FBF7E1FC0022774BFCF790
:1048880021F910B34FF000096E4B83F80090FFF741
:104898008FFADFF8B481404601F078F80520FDF77B
:1048A800D7FE404649464A4601F050F840466C4912
:1048B80001F056F840464946012201F047F84046C3
:1048C800684901F04DF8FFF74DFA674B1B88674AB6
:1048D800A2FB031252094FF4FA7101FB12339BB287
:1048E8001BBB5D4B1B7803BB564B1B78EBB9FFF723
:1048F800D1F9D0B14FF4FA70FDF7AAFEFFF7E0F94D
:10490800DFF84481404600210A4601F01FF840467E
:10491800574901F025F80022474B1A604FF47A7086
:10492800FDF796FE01224C4B1A704F4B1B88514ADB
:10493800A2FB03125209642101FB12339BB2002B24
:1049480040F0AD804C4B1B78012B04D13D4B1B78BC
:10495800002B00F0A480404B1B78DBB9DFF8E8801F
:1049680040460421002200F0F1FF4FF00209CDF883
:104978000090404632463B4601F03CF840460A214A
:10498800002200F0E3FFCDF80090404622462B4677
:1049980001F030F82C4C20460421012200F0D6FF0B
:1049A800364B1868FBF7AAFD02460B460125009511
:1049B800204601F01FF820460B212A4600F0C6FFCA
:1049C8002F4B18680021FCF7CBFB20B12C4B1C683F
:1049D80004F1004401E02A4B1C682A4B18680021A6
:1049E800FCF7BEFB20B1274B196801F1004101E03B
:1049F800244B19682046FCF7D1FB68B1204B186896
:104A08000021FCF7ADFB20B11D4B186800F10040F8
:104A18003CE01B4B186839E01A4B18680021FCF77A
:104A28009FFB88B3174B186800F100402EE000BFC9
:104A380000000000000495400400002098000020B9
:104A4800A000002094000020B8030020D85D0008D2
:104A5800E05D0008E45D0008760000200000E03F0B
:104A6800E85D0008F85D000878000020D34D62106A
:104A7800085E00081F85EB51B600002020000020CA
:104A8800AC000020A80000202F4B1868FBF736FD6B
:104A980002460B46022100912C4800F0ABFF2C4B3C
:104AA8001A8801321A802B4B1C6820464FF084412B
:104AB800FCF756FB38B1284B1B681333262B02D85A
:104AC800FFF750F922E020462449FCF749FB60B182
:104AD80020464FF08441FCF761FB30B10522204BA2
:104AE8001A7006221F4B1A7010E01B4B1B6813F13B
:104AF800320F06DA05221A4B1A700122194B1A7066
:104B080004E00023164A1370164A13708AEAEA73FF
:104B1800A3EBEA73322B05DC029B002BB8BF5B4288
:104B2800322B03DD0022104B1A6003E00E4B1A688B
:104B380001321A600C4B1A680C4B9A427FF6A8AAED
:104B4800FFF710F9FFF7A4BAA8000020B803002067
:104B58007800002020000020740400200000044297
:104B68009C000020800000205C04002000710200EE
:104B78002DE9F8430222704B5A60704B1B68B3F55D
:104B88007A7F3BDA01336D4A13606D4B998889B29D
:104B98006C4A1068014401EBD17149101160D98841
:104BA80089B2694A1068014401EBD171491011605A
:104BB800198889B2654A1068014401EBD17149101E
:104BC8001160598889B2624A1068014401EBD171B9
:104BD80049101160598989B25E4A1068014401EB95
:104BE800D171491011601A8992B25B4B19680A4455
:104BF80002EBD27252101A60BDE8F883574B1E6858
:104C0800574BA3FB06139B094FF47A7202FB1363FD
:104C180013BB544F3868FBF771FC41A3D3E9002359
:104C2800FBF7C0FC04460D46454B988980B2FCF75B
:104C3800A1F84D49FCF7F6F8FBF760FC3AA3D3E975
:104C48000023FBF7AFFC02460B4620462946FBF73C
:104C5800F7FAFBF789FF3860394B588980B23D4B2A
:104C68001B68C01AFBF738FC31A3D3E90023FBF714
:104C780099FCFBF779FF04463C4B18600021FCF7D0
:104C88006FFA28B120463A49FCF76AFA60B904E09D
:104C980020463849FCF782FA30B9374B1B68052B98
:104CA80002D8364B1B782BB9354B5A6C22F400428C
:104CB8005A6404E0324B5A6C42F400425A64204B66
:104CC800188980B2244B1B68C01AFBF705FC18A38F
:104CD800D3E90023FBF766FCFBF746FF0446294BA4
:104CE80018600021FCF73CFA28B120462049FCF75F
:104CF80037FA68B904E020461E49FCF74FFA38B97C
:104D08001D4B1B68052B03D81C4B1B78002B3DD172
:104D18001D4B5A6C22F400425A643CE0AFF3008009
:104D2800AE47E17A14AEEF3F7B14AE47E17A843F99
:104D38007B14AE47E17A943F000002407C000020DB
:104D4800E002002014000020100000201C000020B9
:104D5800180000202400002028000020A4000020C3
:104D6800D34D62102000002017B9CE3CA8000020C7
:104D7800000070C100007041040000209400002071
:104D880000340140AC000020002C01408E4B5A6CCE
:104D980042F400425A648D4B9A6812F0200F14BFF7
:104DA80000220122996811F0400F14BF002101214F
:104DB8009B6813F0800F14BF00200120844B9C686F
:104DC80014F4806F14BF002501259C6814F4006F4B
:104DD80014BF002701279B6813F4805F01EB400391
:104DE80002EB43037B4CE25C7B4B1A601A6802F1CE
:104DF80002021A601868794981FB0082A2EBE0720E
:104E080002EB42024FEA4202C2EB00021A600CBFF8
:104E1800022200223A4405EB4202A05C704A10606C
:104E2800106802301060106881FB0091A1EBE071FE
:104E380001EB41014900411A11601B68694A9088D9
:104E480080B269490968441AD18889B267480268FA
:104E58008A1A052B18D8DFE803F003070A0D101388
:104E6800A21A634B1A6012E0614B1C600FE0604BA2
:104E78001C600CE05E4B1A6009E05D4B1A6006E0AE
:104E8800121B5B4B1A6002E00022594B1A60013674
:104E9800584B1E60584B1B68ABB15849A1FB062103
:104EA800090B574A12680132B1FBF2F002FB1012EB
:104EB8004AB9B6FBF3F203FB12664EB9514810210A
:104EC800FDF7FAFA04E04F4810210022FDF7EEFA48
:104ED8004D4B1A68404B1B68052B1AD8DFE803F0C6
:104EE80003070B0E111515465242002614E05642D0
:104EF8001546002210E0564200250DE055420026D6
:104F08000AE055421646002206E01646524200259F
:104F180002E00022154616463C4B1868304B1B68C9
:104F2800052B1ED8DFE803F003080D1115190746F5
:104F380040424FF0000C17E0C0F1000C074600207B
:104F480012E0C0F1000C00270EE047424FF0000CC1
:104F58000AE047428446002006E084464042002793
:104F680002E0002007468446274B1968002951DDD6
:104F7800274B1968184B1C680534184B83FB04939E
:104F8800A3EBE47303EB43035B00E31A052B70D830
:104F9800DFE803F003070B0E11150B464942002406
:104FA8006CE04C420B46002168E04C42002365E06F
:104FB8004B42002462E04B420C4600215EE00C4666
:104FC800494200235AE000BF002C0140000C014078
:104FD800001001401C5E000888000020ABAAAA2A25
:104FE80090000020E00200201400002010000020A3
:104FF800B0000020A40000209C0000205917B7D161
:10500800800000200008014098000020A000002037
:1050180084000020784B19684B42784C246804F1CE
:105028000108774C84FB0894A4EBE87404EB44046F
:105038006400C4EB0804052C04D8DFE804F01E075C
:105048000A0E131700210B460C4617E00C460021E8
:1050580014E00C461946002310E01C460B46214676
:1050680000240BE01C460B46002107E01C460023E9
:1050780004E000210B460C4600E0002426441D44B1
:1050880001EB02085F4B1B68002B2ADD5E4B1A6898
:105098005E4B1C6805345A4B83FB0493A3EBE47303
:1050A80003EB43035B00E31A052B47D8DFE803F063
:1050B80003070B0E111513465242002143E05142DB
:1050C800134600223FE0514200233CE053420021B6
:1050D80039E053421146002235E01146524200237E
:1050E80031E0494B1A68534248490C680134444935
:1050F80081FB0491A1EBE47101EB41014900611AC4
:10510800052904D8DFE801F01E070A0E131700224C
:105118001346114617E01146002214E011461A46BC
:10512800002310E0194613460A4600210BE01946F1
:105138001346002207E01946002304E00022134624
:10514800114600E0002161443B44024406F57A76AA
:1051580040F2C670864203DC0A2EB8BF0A2601E078
:1051680040F2C6762A48466305F57A7540F2C6705D
:10517800854203DC0A2DB8BF0A2501E040F2C67556
:105188002348856308F57A7440F2C670844203DCCC
:105198000A2CB8BF0A2401E040F2C6741C48C46354
:1051A80001F57A7140F2C670814203DC0A29B8BF62
:1051B8000A2101E040F2C6711648416303F57A738B
:1051C80040F2C6718B4203DC0A2BB8BF0A2301E008
:1051D80040F2C6730F498B6302F57A7240F2C673C8
:1051E8009A4203DC0A2AB8BF0A2201E040F2C672DA
:1051F800084BDA63BDE8F8838400002088000020AB
:10520800ABAAAA2AA00000208C0000209000002051
:1052180000340140002C0140074A4FF6FF7104E0BA
:1052280003889BB28B4204D104309042F8D9012004
:1052380070470020704700BFFF870008134B1B888A
:1052480099B2134B1B889BB278B1012811D12BB9A5
:105258004EF6EE6399420ED10020704769B94EF6BA
:10526800EE6293420BD14020704751B15BB94020A8
:1052780070470020704740207047AB2070470020DF
:10528800704700207047AB20704700BF00800008BF
:1052980000800108F8B507460E460120FFF7CEFF4B
:1052A800AB281FD000F580341034E402C3020E4D41
:1052B8001D4413E02368B3F1FF3F0ED101202146BE
:1052C800B2B20023FCF74EF800B1F8BD0120A11CD2
:1052D800BAB20023FCF746F8F8BD0434AC42E9D36F
:1052E8008020F8BDAB20F8BDFF87000800B587B067
:1052F8000023059301931248039001230493FFF7B9
:105308008BFF20B901A805A9FCF76AFF88B901201D
:105318000B4900220023FCF725F858B909480390E7
:10532800FFF77AFF38B901A805A9FCF759FF20B99A
:1053380003E002E001E00020FFE707B05DF804FBAE
:10534800008000080080010870B505460E46002060
:10535800FFF774FFAB2813D0C2020A4B13440A4C60
:10536800144409E01A8892B2AA4204D133F8023CE4
:105378003380002070BD043B9C42F3D3012070BDF4
:10538800AB2070BDFE870008028000082DE9F043BD
:1053980087B000210591954A13889BB294480088EC
:1053A80080B201910392012204924EF6EE6293427A
:1053B8003AD04FF6FF72934203D0002B40F0F780AB
:1053C8009CE078B98948FFF727FF0446002840F099
:1053D800F38001A805A9FCF703FF002800F001816C
:1053E8000446FEE04EF6EE63984216D17F48FFF77A
:1053F80013FF38B901A805A9FCF7F2FE04460028F6
:1054080040F0EF8001207A4900220023FBF7AAFF31
:105418000446002800F0D280E3E0FFF767FF044667
:10542800002800F0CD80DCE0F0B146E0B8F80030AC
:105438009BB22C4637F81500834200D1AEB233B286
:105448009C420ED04946FFF77FFF012809D037F864
:105458001400B9F80010FFF71DFF0446002840F0BB
:10546800C0800135ADB207E04FF6FF760025DFF8C2
:105478008881604FDFF88491022DD7D901205B49DC
:1054880000220023FBF76EFF0446002840F0A980A5
:10549800002301935648039001230493FFF7BCFEB1
:1054A8000446002840F08E8001A805A9FCF798FE64
:1054B800002800F09680044693E04FF6FF73984268
:1054C80016D14B480390FFF7A7FE38B901A805A9E4
:1054D800FCF786FE0446002840F0838001204349FB
:1054E80000220023FBF73EFF044600286CD078E03A
:1054F800FFF7FCFE0446002868D072E028B9FFF7E1
:10550800F5FE0446002863D06BE04FF6FF7398421F
:105518002AD137480390FFF77FFE0446002859D167
:1055280001A805A9FCF75CFE00285AD0044658E0FB
:10553800B8F800309BB2254637F81400834200D1F2
:10554800A6B233B29D420CD04946FFF7FDFE0128B2
:1055580007D037F81500B9F80010FFF79BFE0028B0
:105568003AD10134A4B207E04FF6FF760024DFF801
:105578009080204FDFF88490022CD9D901201C4953
:1055880000220023FBF7EEFE044650BB00230193E4
:105598001648039001230493FFF73EFE0446E8B93A
:1055A80001A805A9FCF71CFED8B1044619E0FFF7CD
:1055B8009DFE0446A0B114E0002412E0002410E08F
:1055C80000240EE000240CE000240AE0002408E097
:1055D800002406E0002404E0044602E0002400E081
:1055E8000024204607B0BDE8F08300BF0080000813
:1055F800008001080800002006800008B400002090
:10560800068001082DE9F04786B005460C460020C3
:105618000590FFF713FE402804D0002840D1234FFF
:10562800234E01E0224F214E012031464EF6EE6214
:105638000023FBF797FE00B135E028462146FFF727
:1056480029FE78BB0024DFF86C80DFF86C9011E04D
:1056580038F81400A8420BD04946FFF775FE012818
:1056680006D038F81400B9F80010FFF713FED0B9C7
:105678000134A4B2022CEBD9002301930397012330
:10568800049301A805A9FCF7ABFD00B10BE00120CC
:10569800314600220023FBF765FE00B103E002E07B
:1056A800AB2000E0FFE706B0BDE8F0870080000807
:1056B8000080010808000020B400002038B5054625
:1056C8000C46FFF7E7FD802803D128462146FFF75F
:1056D80099FF38BD08B50246084B1B784BB94030D6
:1056E80092F8341000F0B0FA28B10120034B18707A
:1056F80008BD012008BD002008BD00BFB60000207D
:1057080008B559B1836B53F82230012202FA03F32A
:1057180090F83420134380F834300BE0836B53F84F
:105728002230012202FA03F390F8342022EA03031C
:1057380080F83430FFF7CEFF08BD00BF08B501F090
:1057480001010722FFF7DCFF08BD00BF08B511F013
:10575800010F0AD0836B1B68012202FA03F390F849
:105768003420134380F834300AE0836B1B6801222D
:1057780002FA03F390F8342022EA030380F8343065
:1057880011F0020F0AD0836B5B68012202FA03F35F
:1057980090F83420134380F834300AE0836B5B6858
:1057A800012202FA03F390F8342022EA030380F876
:1057B800343011F0040F0AD0836B9B68012202FA7F
:1057C80003F390F83420134380F834300AE0836BF5
:1057D8009B68012202FA03F390F8342022EA0303BB
:1057E80080F8343011F0080F0AD0836BDB6801228F
:1057F80002FA03F390F83420134380F834300AE0B7
:10580800836BDB68012202FA03F390F8342022EA62
:10581800030380F83430FFF75DFF08BD10B5044678
:1058280000210622FFF76CFF204600210422FFF723
:1058380067FF204601210522FFF762FF204601216C
:105848000622FFF75DFF204600210622FFF758FFDA
:10585800204601210622FFF753FF20460021062299
:10586800FFF74EFF204600210522FFF749FF0020E1
:1058780010BD00BF00B583B00DF10701FFF7CEFFE3
:1058880003B05DF804FB00BF38B504460D46174B5E
:105898001B784BBB00210622FFF732FF2046002170
:1058A8000422FFF72DFF20462909FFF74FFF204666
:1058B80001210622FFF724FF204600210622FFF7D8
:1058C8001FFF20462946FFF741FF204601210622F7
:1058D800FFF716FF204600210622FFF711FF20469A
:1058E800FFF7C8FF002038BD012038BDB6000020F2
:1058F80038B504460D4600210622FFF701FF204671
:1059080001210422FFF7FCFE20462909FFF71EFFAC
:10591800204601210622FFF7F3FE20460021062239
:10592800FFF7EEFE20462946FFF710FF204601212B
:105938000622FFF7E5FE204600210622FFF7E0FEDB
:105948002046FFF797FF002038BD00BF08B501EBE0
:10595800821161F07F01C9B2FFF796FF08BD00BF51
:1059680070B506460D4649B90EE03046FFF782FF8E
:105978003046295DFFF7BCFF013400E000244F2CBE
:1059880002DC2B5D002BF0D1002070BD08B5012191
:10599800FFF77AFF08BD00BF08B501224270827880
:1059A800520042F00C02D2B2C1781143FFF76CFFEB
:1059B80008BD00BF10B58AB000238DF82430012A35
:1059C80000D80A2209ACB1FBF2F303FB1211C9B2E9
:1059D800013C092902D83031C9B201E03731C9B2D6
:1059E80021701946002BEED12146FFF7B9FF0AB006
:1059F80010BD00BF2DE9F84F814616461F469DF899
:105A080028B01046194600220023FBF73DF830B1B4
:105A180048463349FFF7A4FF07F100431F464FF0FC
:105A2800000800222F4B00242F4D0BE0104619468A
:105A380022462B46FAF7E0FE02460B4608F101081B
:105A48005FFA88F8D845F1D330463946FAF7F8FBBB
:105A580004460D46FBF768F80646FAF72DFD0246A0
:105A68000B4620462946FAF7E9FB04460D46484608
:105A780031460A22FFF79EFFBBF1000F21D04846AE
:105A88001A49FFF76DFF1CE02046294632463B467F
:105A9800FAF788FD04460D46FBF71EF8834648468C
:105AA80059465246FFF786FF5846FAF715FD024653
:105AB8000B4620462946FAF7C1FB04460D46C34665
:105AC80003E00026084F4FF00A0A0BF1FF385FFA8F
:105AD80088F8BBF1000FD7D10020BDE8F88F00BFD0
:105AE800245E00080000E03F00002440285E000813
:105AF80008B5490041F00401C9B21143FFF7C4FEDB
:105B080008BD00BF10B50446012343700023C370CD
:105B1800837090F83C30002B40F08A80464B8363BA
:105B2800403000F08BF8002840F0848020460021A7
:105B38000422FFF7E5FD204600210522FFF7E0FDDE
:105B4800204600210622FFF7DBFD20460321FFF750
:105B5800FDFD204601210622FFF7D2FD0120FCF7BA
:105B680077FD204600210622FFF7CAFD0520FCF735
:105B78006FFD20460321FFF7E9FD2046012106229B
:105B8800FFF7BEFD0120FCF763FD20460021062239
:105B9800FFF7B6FD0120FCF75BFD20460321FFF768
:105BA800D5FD204601210622FFF7AAFD0120FCF7BA
:105BB8004FFD204600210622FFF7A2FD0120FCF739
:105BC80047FD20460221FFF7C1FD2046012106229C
:105BD800FFF796FD0120FCF73BFD20460021062239
:105BE800FFF78EFD0120FCF733FD2178C900C9B20B
:105BF800204641F02001FFF747FEA3785B0043F001
:105C08000803DBB2E17820461943FFF73DFE204642
:105C1800FFF7BCFE204601210022FFF769FF20465E
:105C2800FFF7BAFE20460121FFF788FD002010BDCE
:105C3800012010BD012010BD2C000020037803F0C6
:105C4800070303700020704700B585B004AA02F866
:105C5800011D034613F8081B4900406800901846C8
:105C680041F040010123FDF7BBF908B1012000E034
:105C7800002005B05DF804FB704700BFFEE700BFD9
:105C8800FEE700BFFEE700BFFEE700BF704700BFAA
:105C9800704700BF704700BF08B5FCF7CBFCFCF7A6
:105CA80077FA08BD002100F004B80D4B5B5843504B
:105CB80004310C480C4B42189A42FFF4F6AF0B4AD9
:105CC80000F003B8002342F8043B094B9A42FFF462
:105CD800F9AFFDF71BFC00F00FF8FEF7CDF87047A1
:105CE800345E0008000000204C0000205000002016
:105CF80088040020FFF7FEBF70B50E4B0E4D002440
:105D0800ED1AAD101E46AC4204D056F82420904738
:105D18000134F8E700F020F8084D094B0024ED1A8B
:105D2800AD101E46AC4204D056F8242090470134EA
:105D3800F8E770BD2C5E00082C5E0008305E000895
:105D48002C5E000810B50023934203D0CC5CC454E9
:105D58000133F9E710BD0000F8B500BFF8BC08BC76
:105D68009E467047F8B500BFF8BC08BC9E46704711
:105D780002030405060708090A0B0C0D0E0F101084
:105D880001020000000000000000000001020304FE
:105D98000607080900000000010203045472616E3E
:105DA80073704F747465722056322E3100000000F3
:105DB800496E697469616C697A696E672E2E2E0066
:105DC8004261743A000000005600000041000000E3
:105DD8004C656E3A000000006D2800006D29000037
:105DE800456D657267656E6379204F6666210000B0
:105DF8004B656570657220746F20666173742E0040
:105E08004E756E636875636B20436F6E74726F6C4A
:105E18000000000000000201040503002D0000003E
:045E28002E00000048
:045E2C000D0200085B
:045E3000E90100087C
:105E340000A24A04640000003713000000000000C0
:105E4400D0070000D0070000D0070000D0070000F2
:105E540000002042D0070000D0070000040000002A
:105E6400050000000600000007000000000000001C
:0C5E74000100000002000000030000001C
:0400000508005CADE6
:00000001FF
